BL51 BANKED LINKER/LOCATER V6.22.2.0                                                    07/03/2023  14:57:11  PAGE 1


BL51 BANKED LINKER/LOCATER V6.22.2.0, INVOKED BY:
C:\KEIL_V5\C51\BIN\BL51.EXE .\Release\system_FE81001.obj, .\Release\STARTUP.obj, .\Release\main.obj TO .\Release\Sample_
>> DrvSDM_MultiB REGFILE (.\Release\Sample_DrvSDM_MultiB.ORC) PRINT (.\Sample_DrvSDM_MultiB.m51) RAMSIZE (256) CODE (0X0
>> 000-0X1FFF) XDATA (0X8000-0X87FF)


MEMORY MODEL: SMALL


INPUT MODULES INCLUDED:
  .\Release\system_FE81001.obj (SYSTEM_FE81001)
  .\Release\STARTUP.obj (?C_STARTUP)
  .\Release\main.obj (MAIN)
  C:\KEIL_V5\C51\LIB\C51S.LIB (?C_INIT)
  C:\KEIL_V5\C51\LIB\C51S.LIB (?C_IBP)


LINK MAP OF MODULE:  .\Release\Sample_DrvSDM_MultiB (SYSTEM_FE81001)


            TYPE    BASE      LENGTH    RELOCATION   SEGMENT NAME
            -----------------------------------------------------

            * * * * * * *   D A T A   M E M O R Y   * * * * * * *
            REG     0000H     0008H     ABSOLUTE     "REG BANK 0"
            DATA    0008H     0003H     UNIT         ?DT?MAIN
            DATA    000BH     0002H     UNIT         ?DT?DELAY?MAIN
            DATA    000DH     0001H     UNIT         ?DT?SDMISR?MAIN
            DATA    000EH     0001H     UNIT         ?C?LIB_DATA
            IDATA   000FH     0001H     UNIT         ?STACK

            * * * * * * *   C O D E   M E M O R Y   * * * * * * *
            CODE    0000H     0003H     ABSOLUTE     
            CODE    0003H     001CH     UNIT         ?PR?DELAY?MAIN
            CODE    001FH     0006H     UNIT         ?C_INITSEG
            CODE    0025H     0001H     UNIT         ?PR?SYSTEMINIT?SYSTEM_FE81001
                    0026H     0005H                  *** GAP ***
            CODE    002BH     0003H     ABSOLUTE     
            CODE    002EH     009DH     UNIT         ?C_C51STARTUP
            CODE    00CBH     0096H     UNIT         ?PR?SDMCONFIG?MAIN
            CODE    0161H     0053H     UNIT         ?PR?IOCONFIG?MAIN
            CODE    01B4H     004EH     UNIT         ?PR?ANACCONFIG?MAIN
            CODE    0202H     0040H     UNIT         ?PR?SDMISR?MAIN
            CODE    0242H     0038H     UNIT         ?PR?CLKCONFIG?MAIN
            CODE    027AH     0018H     UNIT         ?PR?MAIN?MAIN



OVERLAY MAP OF MODULE:   .\Release\Sample_DrvSDM_MultiB (SYSTEM_FE81001)


SEGMENT
  +--> CALLED SEGMENT
---------------------
?C_C51STARTUP
  +--> ?PR?MAIN?MAIN
  +--> ?C_INITSEG

BL51 BANKED LINKER/LOCATER V6.22.2.0                                                  07/03/2023  14:57:11  PAGE 2


?PR?MAIN?MAIN
  +--> ?PR?CLKCONFIG?MAIN
  +--> ?PR?IOCONFIG?MAIN
  +--> ?PR?ANACCONFIG?MAIN
  +--> ?PR?SDMCONFIG?MAIN
  +--> ?PR?DELAY?MAIN



SYMBOL TABLE OF MODULE:  .\Release\Sample_DrvSDM_MultiB (SYSTEM_FE81001)

  VALUE           TYPE          NAME
  ----------------------------------

  -------         MODULE        SYSTEM_FE81001
  C:0000H         SYMBOL        _ICE_DUMMY_
  C:0025H         PUBLIC        SystemInit
  -------         PROC          SYSTEMINIT
  C:0025H         LINE#         38
  C:0025H         LINE#         39
  C:0025H         LINE#         41
  -------         ENDPROC       SYSTEMINIT
  -------         ENDMOD        SYSTEM_FE81001

  -------         MODULE        ?C_STARTUP
  C:002EH         SEGMENT       ?C_C51STARTUP
  I:000FH         SEGMENT       ?STACK
  C:0000H         PUBLIC        ?C_STARTUP
  D:00E0H         SYMBOL        ACC
  D:00F0H         SYMBOL        B
  D:0083H         SYMBOL        DPH
  D:0082H         SYMBOL        DPL
  N:0001H         SYMBOL        IBPSTACK
  N:0100H         SYMBOL        IBPSTACKTOP
  N:0080H         SYMBOL        IDATALEN
  C:0031H         SYMBOL        IDATALOOP
  N:0000H         SYMBOL        PBPSTACK
  N:0100H         SYMBOL        PBPSTACKTOP
  N:0000H         SYMBOL        PDATALEN
  N:0000H         SYMBOL        PDATASTART
  N:0000H         SYMBOL        PPAGE
  N:0000H         SYMBOL        PPAGEENABLE
  D:00A0H         SYMBOL        PPAGE_SFR
  D:0081H         SYMBOL        SP
  C:002EH         SYMBOL        STARTUP1
  N:0000H         SYMBOL        XBPSTACK
  N:0000H         SYMBOL        XBPSTACKTOP
  N:0800H         SYMBOL        XDATALEN
  C:003CH         SYMBOL        XDATALOOP
  N:8000H         SYMBOL        XDATASTART
  C:0000H         LINE#         126
  C:002EH         LINE#         133
  C:0030H         LINE#         134
  C:0031H         LINE#         135
  C:0032H         LINE#         136
  C:0034H         LINE#         140
  C:0037H         LINE#         141
BL51 BANKED LINKER/LOCATER V6.22.2.0                                                  07/03/2023  14:57:11  PAGE 3


  C:0039H         LINE#         145
  C:003BH         LINE#         147
  C:003CH         LINE#         148
  C:003DH         LINE#         149
  C:003EH         LINE#         150
  C:0040H         LINE#         151
  C:0042H         LINE#         170
  C:0045H         LINE#         185
  C:0048H         LINE#         196
  -------         ENDMOD        ?C_STARTUP

  -------         MODULE        MAIN
  C:0000H         SYMBOL        _ICE_DUMMY_
  D:00A8H         PUBLIC        IE
  C:0003H         PUBLIC        delay
  D:00B8H         PUBLIC        IP
  C:027AH         PUBLIC        main
  D:0098H         PUBLIC        SCON
  C:0242H         PUBLIC        CLKConfig
  D:0088H         PUBLIC        TCON
  D:0080H         PUBLIC        SfrPA
  C:00CBH         PUBLIC        SDMConfig
  D:0090H         PUBLIC        SfrPB
  D:00A0H         PUBLIC        SfrPC
  D:00B0H         PUBLIC        SfrPD
  D:0008H         SYMBOL        raw_data
  C:0202H         PUBLIC        SDMISR
  D:00C8H         PUBLIC        T2CON
  C:01B4H         PUBLIC        ANACConfig
  C:0161H         PUBLIC        IOConfig
  D:00D0H         PUBLIC        PSW
  -------         PROC          DELAY
  -------         DO            
  D:000BH         SYMBOL        i
  -------         ENDDO         
  C:0003H         LINE#         35
  C:0003H         LINE#         36
  C:0003H         LINE#         39
  C:001EH         LINE#         40
  -------         ENDPROC       DELAY
  -------         PROC          SDMISR
  -------         DO            
  D:000DH         SYMBOL        int_stat
  -------         ENDDO         
  C:0202H         LINE#         52
  C:020FH         LINE#         54
  C:0216H         LINE#         56
  C:021CH         LINE#         59
  C:0223H         LINE#         60
  C:022AH         LINE#         61
  C:0231H         LINE#         64
  C:0237H         LINE#         65
  -------         ENDPROC       SDMISR
  -------         PROC          SDMCONFIG
  C:00CBH         LINE#         77
  C:00CBH         LINE#         78
  C:00CBH         LINE#         82
BL51 BANKED LINKER/LOCATER V6.22.2.0                                                  07/03/2023  14:57:11  PAGE 4


  C:00D0H         LINE#         85
  C:00E1H         LINE#         88
  C:00F2H         LINE#         91
  C:00FDH         LINE#         94
  C:0108H         LINE#         97
  C:011EH         LINE#         100
  C:013FH         LINE#         103
  C:014AH         LINE#         106
  C:0155H         LINE#         109
  C:0160H         LINE#         111
  -------         ENDPROC       SDMCONFIG
  -------         PROC          ANACCONFIG
  C:01B4H         LINE#         123
  C:01B4H         LINE#         124
  C:01B4H         LINE#         126
  C:01BFH         LINE#         127
  C:01CAH         LINE#         128
  C:01D5H         LINE#         131
  C:01E0H         LINE#         134
  C:01EBH         LINE#         137
  C:01F6H         LINE#         140
  C:0201H         LINE#         142
  -------         ENDPROC       ANACCONFIG
  -------         PROC          IOCONFIG
  C:0161H         LINE#         153
  C:0161H         LINE#         154
  C:0161H         LINE#         156
  C:0182H         LINE#         159
  C:01A3H         LINE#         162
  C:01A8H         LINE#         163
  C:01AEH         LINE#         164
  C:01B3H         LINE#         165
  -------         ENDPROC       IOCONFIG
  -------         PROC          CLKCONFIG
  C:0242H         LINE#         177
  C:0242H         LINE#         178
  C:0242H         LINE#         180
  C:024DH         LINE#         183
  C:0258H         LINE#         184
  C:0263H         LINE#         187
  C:0279H         LINE#         188
  -------         ENDPROC       CLKCONFIG
  -------         PROC          MAIN
  C:027AH         LINE#         200
  C:027AH         LINE#         201
  C:027AH         LINE#         202
  C:027DH         LINE#         203
  C:0280H         LINE#         205
  C:0283H         LINE#         206
  C:0286H         LINE#         209
  C:028CH         LINE#         211
  C:028FH         LINE#         213
  -------         ENDPROC       MAIN
  -------         ENDMOD        MAIN

  -------         MODULE        ?C_IBP
  D:000EH         PUBLIC        ?C_IBP
BL51 BANKED LINKER/LOCATER V6.22.2.0                                                  07/03/2023  14:57:11  PAGE 5


  -------         ENDMOD        ?C_IBP



FUNCTION REGISTER MASKS


FUNCTION . . . . . REG MASK
---------------------------

ANACCONFIG . . . . @0xe301
CLKCONFIG. . . . . @0xe301
DELAY. . . . . . . @0xf000
IOCONFIG . . . . . @0xe301
MAIN . . . . . . . @0xf301
SDMCONFIG. . . . . @0xe301
SDMISR . . . . . . @0xa301
SYSTEMINIT . . . . @0x8000

*** WARNING L16: UNCALLED SEGMENT, IGNORED FOR OVERLAY PROCESS
    SEGMENT: ?PR?SYSTEMINIT?SYSTEM_FE81001

Program Size: data=16.0 xdata=0 code=653
LINK/LOCATE RUN COMPLETE.  1 WARNING(S),  0 ERROR(S)
